:020000040000FA
:0600000000008A01B12995
:08000800F000030E8301F1007A
:100010008B1029108513721D0F2876207211291D4F
:1000200045282910A10A0A302106031D2A28A1010A
:10003000A20A0A302206031D2A28A201A30A0A30B6
:100040002306031D2A28A301A40A0A302406031D3F
:100050002A28A40121082E06031D622822082F0643
:10006000031D622823083006031D62282408310678
:10007000031D6228A91C41282914851772150B122B
:100080006228762029148517622800000930A10310
:10009000A11F5728A100A203A21F5728A200A30353
:1000A000A31F5728A300A403A41F5728A4002108B6
:1000B000220423042404031D6228291485177215C1
:1000C000A9180B12710E8300F00E700E0900820742
:1000D0003F3406345B344F3466346D347D3407343A
:1000E0007F346F340034403450341834B208031D68
:1000F00008008B100B16721129108513291D8528F5
:10010000A101A201A301A40108002E08A1002F084B
:10011000A2003008A3003108A40008000C30A90692
:1001200008000230A9068B100B1608002108672072
:10013000A50022086720A60023086720A70024083E
:100140006720A800F21C0800B208031D08000A304E
:100150006720A408031D0800A800A308031D0800C9
:10016000A700A2080319A600080005088039850029
:100170001030AA0C0318AA002A18250DAA18260D5B
:100180002A19270DAA19280D2A1A290D7218FF3AC3
:100190008600050880392A04850000000000000060
:1001A000051BAB042A09051FAB052A1C0800A00B80
:1001B00008000530A0002C082B062B05AD002B08ED
:1001C000AC00F21508000B120B12B208031DF12847
:1001D0000B30A400A300A200A101B20A21308400C8
:1001E00008000408243A0319F828840A800108004A
:1001F0002108AE002208AF002308B0002408B10097
:10020000A101A201A301A401B2019C2176208B10BF
:100210000B160800B20803190800800A00080A3A01
:100220000319800108001030B20025210C1D162989
:100230000C11B520F21D1629F2112D1A2521AD1D24
:100240001629B2015621762008000830B20C031896
:10025000B20032184C29B2184229321939293029F2
:10026000F21072120D30A4000030A300A200A10011
:100270009628F21072160C30A4000030A300A200E1
:10028000A1009628F21472120D30A4000A30A300C7
:10029000A2000030A1009628F21472160C30A400BF
:1002A0000A30A300A2000030A100962800008312AB
:1002B00003178D0172085F218312031308000000E9
:1002C000831203130D12831203178C008316031776
:1002D0008C130C158B138B1B6A2955308D00AA309B
:1002E0008D008C140C118B17831203130D1E7629AD
:1002F0008312031708000000831203178D00831672
:1003000003178C130C14831203170C0883120313A6
:10031000080003017B211239F200080000000130BF
:100320007B21B10002307B21B00003307B21AF0084
:1003300004307B21AE000800000001308312031757
:100340008D00831203133108AA213008AA212F0837
:10035000AA212E085F21831203178D0A831203132B
:10036000080083018601831670308F000030810001
:100370009B0101308600603085008312FF308600CB
:10038000083085008020A9010030AE00AF00B00029
:10039000B1002915A911FF30AB00AC000530A00059
:1003A000043092000B309700D03095000730960053
:1003B0000130900089218E2172141030AA00051B93
:1003C0001321B2018316721A011783120B168B17B1
:1003D0000C19EB21E8290C119620B520F21D08001C
:1003E000F2112D188E20AD1876202D199120AD19FF
:0803F000E3202D1A0A21080088
:02400E00703F01
:02401000FC3F73
:0A420000FF000000000000000000B5
:1042100063006F0075006E0074006500720032006C
:0E4220003000300039002E00610073006D0088
:00000001FF
